:020000040800F2
:1040000000C00020D5710008956F0008976F000868
:10401000996F00089B6F00089D6F0008000000006A
:104020000000000000000000000000009F6F00087A
:10403000A16F000800000000A36F0008A56F000832
:104040001D7200081D7200081D7200081D72000814
:104050001D7200081D7200081D7200081D72000804
:104060001D7200081D7200081D720008A96F00086B
:104070001D7200081D720008B56F0008C16F0008AE
:10408000CD6F0008D96F0008E56F00081D720008A9
:104090001D7200081D7200081D7200081D720008C4
:1040A0001D7200081D7200081D7200081D720008B4
:1040B0001D7200081D7200081D7200081D720008A4
:1040C0001D7200081D7200081D7200081D72000894
:1040D0001D720008017000080D7000081D720008B4
:1040E0001D7200081D7200081D7200081D72000874
:1040F0001D7200081D7200081D720008197000086A
:104100001D7200081D7200081D7200081D72000853
:10411000257000081D720008317000081D7200082B
:104120001D7200081D7200081D7200081D72000833
:10413000000000000000000000000000000000007F
:10414000000000000000000000000000000000006F
:10415000000000000000000000000000000000005F
:10416000000000000000000000000000000000004F
:10417000000000000000000000000000000000003F
:10418000000000000000000000000000000000002F
:10419000000000000000000000000000000000001F
:1041A000000000000000000000000000000000000F
:1041B00000000000000000000000000000000000FF
:1041C00000000000000000000000000000000000EF
:1041D00000000000000000000000000000000000DF
:0441E0005FF8E0F1B3
:1041E80010B5054C237833B9044B13B10448AFF329
:1041F80000800123237010BDDC03002000000000B4
:10420800649F000808B5034B1BB103490348AFF38B
:10421800008008BD00000000E0030020649F000843
:10422800034613F8012B002AFBD1181A01387047EE
:1042380081F0004102E000BF83F0004330B54FEA4F
:1042480041044FEA430594EA050F08BF90EA020FBC
:104258001FBF54EA000C55EA020C7FEA645C7FEA4F
:10426800655C00F0E2804FEA5454D4EB5555B8BF72
:104278006D420CDD2C4480EA020281EA030382EAE3
:10428800000083EA010180EA020281EA0303362D75
:1042980088BF30BD11F0004F4FEA01314FF4801C48
:1042A8004CEA113102D0404261EB410113F0004F5A
:1042B8004FEA03334CEA133302D0524263EB430311
:1042C80094EA050F00F0A780A4F10104D5F1200EAF
:1042D8000DDB02FA0EFC22FA05F2801841F100010A
:1042E80003FA0EF2801843FA05F359410EE0A5F1DE
:1042F80020050EF1200E012A03FA0EFC28BF4CF00F
:10430800020C43FA05F3C01851EBE37101F00045C4
:1043180007D54FF0000EDCF1000C7EEB00006EEBD1
:104328000101B1F5801F1BD3B1F5001F0CD349085B
:104338005FEA30004FEA3C0C04F101044FEA4452B2
:1043480012F5800F80F09A80BCF1004F08BF5FEA39
:10435800500C50F1000041EB045141EA050130BD19
:104368005FEA4C0C404141EB010111F4801FA4F1BC
:104378000104E9D191F0000F04BF01460020B1FA11
:1043880081F308BF2033A3F10B03B3F120020CDA49
:104398000C3208DD02F1140CC2F10C0201FA0CF027
:1043A80021FA02F10CE002F11402D8BFC2F1200C8C
:1043B80001FA02F120FA0CFCDCBF41EA0C01904042
:1043C800E41AA2BF01EB0451294330BD6FEA04048B
:1043D8001F3C1CDA0C340EDC04F11404C4F1200276
:1043E80020FA04F001FA02F340EA030021FA04F388
:1043F80045EA030130BDC4F10C04C4F1200220FADF
:1044080002F001FA04F340EA0300294630BD21FA1C
:1044180004F0294630BD94F0000F83F4801306BFE2
:1044280081F480110134013D4EE77FEA645C18BFD6
:104438007FEA655C29D094EA050F08BF90EA020F6D
:1044480005D054EA000C04BF1946104630BD91EA65
:10445800030F1EBF0021002030BD5FEA545C05D168
:104468004000494128BF41F0004130BD14F58004A7
:104478003CBF01F5801130BD01F0004545F0FE411B
:1044880041F470014FF0000030BD7FEA645C1ABF50
:10449800194610467FEA655C1CBF0B46024650EA87
:1044A800013406BF52EA033591EA030F41F40021B3
:1044B80030BD00BF90F0000F04BF0021704730B539
:1044C8004FF4806404F132044FF000054FF000010E
:1044D80050E700BF90F0000F04BF0021704730B5CF
:1044E8004FF4806404F1320410F0004548BF4042A4
:1044F8004FF000013EE700BF42004FEAE2014FEAF9
:1045080031014FEA02701FBF12F07F4393F07F4FD3
:1045180081F06051704792F0000F14BF93F07F4F05
:10452800704730B54FF4607401F0004521F0004148
:1045380020E700BF50EA010208BF704730B54FF0CE
:1045480000050AE050EA010208BF704730B511F0D3
:10455800004502D5404261EB41014FF4806404F10B
:1045680032045FEA915C3FF4DCAE4FF003025FEA8D
:10457800DC0C18BF03325FEADC0C18BF033202EB15
:10458800DC02C2F1200300FA03FC20FA02F001FA6F
:1045980003FE40EA0E0021FA02F11444C1E600BF0E
:1045A80070B54FF0FF0C4CF4E06C1CEA11541DBFC1
:1045B8001CEA135594EA0C0F95EA0C0F00F0DEF88C
:1045C8002C4481EA030621EA4C5123EA4C5350EA71
:1045D800013518BF52EA033541F4801143F48013C2
:1045E80038D0A0FB02CE4FF00005E1FB02E506F053
:1045F8000042E0FB03E54FF00006E1FB03569CF0A8
:10460800000F18BF4EF0010EA4F1FF04B6F5007FAD
:1046180064F5407404D25FEA4E0E6D4146EB06061F
:1046280042EAC62141EA55514FEAC52040EA5E50A8
:104638004FEACE2EB4F1FD0C88BFBCF5E06F1ED852
:10464800BEF1004F08BF5FEA500E50F1000041EB89
:10465800045170BD06F0004646EA010140EA020036
:1046680081EA0301B4EB5C04C2BFD4EB0C0541EA58
:10467800045170BD41F480114FF0000E013C00F36D
:10468800AB8014F1360FDEBF002001F0004170BD91
:10469800C4F10004203C35DA0C341BDC04F11404AA
:1046A800C4F1200500FA05F320FA04F001FA05F236
:1046B80040EA020001F0004221F0004110EBD37003
:1046C80021FA04F642EB06015EEA430E08BF20EA2F
:1046D800D37070BDC4F10C04C4F1200500FA04F3D2
:1046E80020FA05F001FA04F240EA020001F0004164
:1046F80010EBD37041F100015EEA430E08BF20EAD7
:10470800D37070BDC4F1200500FA05F24EEA020E1E
:1047180020FA04F301FA05F243EA020321FA04F04D
:1047280001F0004121FA04F220EA020000EBD37004
:104738005EEA430E08BF20EAD37070BD94F0000F04
:104748000FD101F00046400041EB010111F4801F38
:1047580008BF013CF7D041EA060195F0000F18BFE9
:10476800704703F00046520043EB030313F4801F25
:1047780008BF013DF7D043EA0603704794EA0C0FDF
:104788000CEA135518BF95EA0C0F0CD050EA4106F5
:1047980018BF52EA4306D1D181EA030101F0004172
:1047A8004FF0000070BD50EA410606BF104619469A
:1047B80052EA430619D094EA0C0F02D150EA0136A6
:1047C80013D195EA0C0F05D152EA03361CBF1046E7
:1047D80019460AD181EA030101F0004141F0FE4186
:1047E80041F470014FF0000070BD41F0FE4141F40A
:1047F800780170BD70B54FF0FF0C4CF4E06C1CEA0A
:1048080011541DBF1CEA135594EA0C0F95EA0C0FBE
:1048180000F0A7F8A4EB050481EA030E52EA033579
:104828004FEA013100F088804FEA03334FF080559A
:1048380045EA131343EA12634FEA022245EA1115C7
:1048480045EA10654FEA00260EF000419D4208BF78
:10485800964244F1FD0404F5407402D25B084FEA25
:104868003202B61A65EB03055B084FEA32024FF4D1
:1048780080104FF4002CB6EB020E75EB030E22BF2E
:10488800B61A754640EA0C005B084FEA3202B6EBEE
:10489800020E75EB030E22BFB61A754640EA5C009D
:1048A8005B084FEA3202B6EB020E75EB030E22BF2D
:1048B800B61A754640EA9C005B084FEA3202B6EB2E
:1048C800020E75EB030E22BFB61A754640EADC00ED
:1048D80055EA060E18D04FEA051545EA16754FEA4F
:1048E80006164FEAC30343EA52734FEAC2025FEA6D
:1048F8001C1CC0D111F4801F0BD141EA00014FF0FC
:1049080000004FF0004CB6E711F4801F04BF0143CC
:104918000020B4F1FD0C88BFBCF5E06F3FF6AFAEE8
:10492800B5EB030C04BFB6EB020C5FEA500C50F178
:10493800000041EB045170BD0EF0004E4EEA1131FB
:1049480014EB5C04C2BFD4EB0C0541EA045170BD02
:1049580041F480114FF0000E013C90E645EA060E46
:104968008DE60CEA135594EA0C0F08BF95EA0C0F74
:104978003FF43BAF94EA0C0F0AD150EA01347FF4BC
:1049880034AF95EA0C0F7FF425AF104619462CE793
:1049980095EA0C0F06D152EA03353FF4FDAE1046F6
:1049A800194622E750EA410618BF52EA43067FF447
:1049B800C5AE50EA41047FF40DAF52EA43057FF4D7
:1049C800EBAE12E74FF0FF3C06E000BF4FF0010CE2
:1049D80002E000BF4FF0010C4DF804CD4FEA410C46
:1049E8007FEA6C5C4FEA430C18BF7FEA6C5C1BD013
:1049F80001B050EA410C0CBF52EA430C91EA030F94
:104A080002BF90EA020F0020704710F1000F91EAF0
:104A1800030F58BF994208BF90422CBFD8176FEABE
:104A2800E37040F0010070474FEA410C7FEA6C5C8C
:104A380002D150EA013C07D14FEA430C7FEA6C5C93
:104A4800D6D152EA033CD3D05DF8040B704700BFBF
:104A58008446104662468C461946634600E000BF0D
:104A680001B5FFF7B7FF002848BF10F1000F01BDDF
:104A78004DF808EDFFF7F4FF0CBF012000205DF8AA
:104A880008FB00BF4DF808EDFFF7EAFF34BF01202F
:104A980000205DF808FB00BF4DF808EDFFF7E0FFC8
:104AA80094BF012000205DF808FB00BF4DF808ED19
:104AB800FFF7CEFF94BF012000205DF808FB00BF80
:104AC8004DF808EDFFF7C4FF34BF012000205DF862
:104AD80008FB00BF4FEA410C7FEA6C5C02D150EA48
:104AE800013C0AD14FEA430C7FEA6C5C02D152EADE
:104AF800033C02D14FF0000070474FF001007047AF
:104B08004FEA410212F5001215D211D56FF47873ED
:104B1800B3EB625212D94FEAC12343F0004343EA90
:104B2800505311F0004F23FA02F018BF404270476B
:104B38004FF00000704750EA013005D111F00040F5
:104B480008BF6FF0004070474FF00000704700BF8B
:104B580038B50E4B054618784FF47A73B3FBF0F36B
:104B68000B4A1068B0FBF3F000F04CFB044658B950
:104B78000F2D09D8024629464FF0FF3000F000FB00
:104B8800044B20461D6038BD012038BD00000020C0
:104B98000802002004000020074A08B51368032013
:104BA80043F01003136000F0D9FA0020FFF7D0FF9C
:104BB80002F046F8002008BD00200240034A044BDA
:104BC80011681B780B441360704700BF180400205D
:104BD80000000020014B1868704700BF180400202F
:104BE80038B50446FFF7F6FF0546631C1EBF044BA5
:104BF8001B78E418FFF7EEFF401B8442FAD838BD53
:104C0800000000207047436A10B59A6A12F0500FEE
:104C18001BD19A6A42F400729A621A68926802F486
:104C28006022B2F5602F0CD11A7B52B99A6A22F42D
:104C380080729A629A6AD2045EBF9A6A42F001024E
:104C48009A621846FFF7DEFF10BD1B6ABDE81040E8
:104C58001B6B1847704708B5406AFFF7FBFF08BD94
:104C68007047036810B55A680446900627D51A6835
:104C7800910724D5A26AD2065EBFA26A42F40072E6
:104C8800A2629A6802F46022B2F5602F10D1227BEA
:104C980072B95A6822F020025A60A36A23F480731A
:104CA800A362A36ADB045EBFA36A43F00103A362A5
:104CB8002046FFF7A7FF6FF0120223681A602368E7
:104CC8005A68100630D51A6851072DD5A26AD2063F
:104CD8005EBFA26A42F40052A2629A6802F4E042FD
:104CE800B2F5E04F0AD05A68500516D49A6802F413
:104CF8006022B2F5602F10D1227B72B95A6822F077
:104D080080025A60A36A23F48053A362A36AD90578
:104D18005EBFA36A43F00103A362204600F01CFAB9
:104D28006FF00C0223681A6023685A6852060DD582
:104D38001B68DB070AD5A36A204643F48033A362C5
:104D4800FFF78EFF6FF0010223681A6010BD7047ED
:104D5800406A08B5836A43F040038362C36A43F03C
:104D68000403C362FFF7F3FF08BD0000002373B517
:104D7800019390F82430012B74D001234D6880F8FA
:104D88002430062D02684FEA85030C6825D82B4489
:104D98001F25566B053B9D4026EA050504FA03F3DB
:104DA8002B435363092C4FEA44038D682FD90726F8
:104DB8002344D1681E3B9E4021EA060105FA03F30D
:104DC8000B43D360A4F11003012B2BD9002300223D
:104DD80080F82420184602B070BD0C2D0BD82B4447
:104DE8001F25166B233B9D4026EA050504FA03F3AD
:104DF8002B431363D6E72B441F25D66A413B9D40BE
:104E080026EA050504FA03F32B43D362CAE707260B
:104E1800116923449E4021EA060105FA03F30B4376
:104E28001361CFE7104B9A4216D193681B02CDD479
:104E38009368102C43F400039360C7D10B4B0C4AC2
:104E48001B68B3FBF2F20A2353430193019B002B27
:104E5800BCD0019B013BF8E7836A43F020038362DF
:104E68000123B4E70223B5E700240140080200202B
:104E780040420F00002373B50193036804469A6803
:104E8800D20702D5002002B070BD9A6842F0010234
:104E98009A60124B124A1B68B3FBF2F30193019B11
:104EA800C3B9FFF797FE064623689D6815F001050C
:104EB800E8D1FFF78FFE801B0228F5D9A36A84F892
:104EC800245043F01003A362E36A012043F0010376
:104ED800E362D8E7019B013BE0E700BF080200203E
:104EE80040420F002DE9D8419046404B02680446E5
:104EF8009A420F4602D03E498A4203D15B6813F4B6
:104F0800702F6ED194F82430012B6CD001232046E9
:104F180084F82430FFF7AEFF064600285DD1A06A6A
:104F2800216820F47060324B20F0010040F480705A
:104F38009942A06204D12D4A536813F4702F3ED1D0
:104F4800A36A23F48013A3624B685A0505D5A36AA4
:104F580023F4405343F48053A362A36A206A13F4F2
:104F6800805318BFE36A3A4618BF23F00603E3628A
:104F7800002384F824301F4B4C3183621E4BC362DC
:104F88001E4B03636FF0020341F84C3C51F8443C5C
:104F980043F4807341F8443C434600F089F92368A0
:104FA8009A6802F46022B2F5602F9A680CBF42F446
:104FB800A00242F480129A603046BDE8D881A36A04
:104FC80043F48013A36253685B0541BFA06A20F4D1
:104FD800405040F48050A062BFE7002384F824309A
:104FE800EAE70126E8E70226E6E700BF00240140D9
:104FF800002801400F4C00085F4C0008594D00087C
:1050080038B5036804469A68D20701D4002038BD31
:105018009A6822F001029A60FFF7DCFD05462368D2
:105028009B68DB07F2D5FFF7D5FD401B0228F6D9B0
:10503800A36A012043F01003A362E36A43F001036B
:10504800E36238BDF8B50446002877D0836A23B9EF
:10505800C36280F8243001F015FE2046FFF7D0FF28
:10506800A36A13F010036BD1002869D1A26A3749EB
:1050780022F4885222F0020242F00202A26294E86C
:1050880024008A42E16904D1B1F5402F08BF4FF4EA
:105098000021267B45EA46052943A568B5F5807FAA
:1050A80035D0012D08BF4FF48073277D012F06D11D
:1050B8007EBBA669013E43EA463343F40063566863
:1050C800B5F5807F26F4694643EA0603536096687F
:1050D8001F4B03EA060343EA0103936001D0012D45
:1050E80020D12369013B1B05D56A25F470052B43A4
:1050F800D3629268174B1340994215D10023E3629B
:10510800A36A23F0030343F00103A362F8BD2B460F
:10511800CBE7A66A46F02006A662E66A46F00106D4
:10512800E662CCE70023DFE7A36A23F0120343F02B
:105138001003A362E36A43F00103E3620120F8BDB0
:10514800A36A43F01003A362F8E700BF003C0140E4
:10515800FDF7E1FFFE0E1FFF70470000074A00023F
:10516800D36800F4E06023F4E0631B041B0C43F0F5
:10517800BF6343F400330343D360704700ED00E09E
:10518800174B30B5DC68C4F30224C4F10703251DAE
:10519800042B28BF0423062D4FF0010598BF0024D7
:1051A80005FA03F303F1FF3388BF033C1940A1401C
:1051B80005FA04F4013C2240002842EA01024FEAC1
:1051C8000212A9BF00F16040064BD2B200F561405F
:1051D800BBBF00F00F00D2B280F800231A5430BDD4
:1051E80000ED00E014ED00E0002808DB012342098F
:1051F80000F01F0003FA00F0014B43F8220070474B
:1052080000E100E00138B0F1807F0AD2F021064BBE
:10521800064A586082F823100020072298601A6016
:1052280070470120704700BF10E000E000ED00E08B
:1052380010B5002832D00168194B1424994225D89A
:10524800184AA3F207430A44B2FBF4F2920002643C
:105258008468C36343680A682343C46822F47F529E
:105268002343046922F030022343446923438469B9
:105278002343C469234313430B600122002380F8AE
:105288002120836380F82030184610BD064B0B445C
:10529800B3FBF4F39B000364044BD9E7012010BD72
:1052A80007040240F8FFFDBFF8FBFDBF0004024001
:1052B800F0B590F82040012C35D0012490F8215009
:1052C80080F82040A5424FF000064FF0020428D194
:1052D80080F82140046886632668076C26F001067A
:1052E8002660C66BBD407560636043680568102B17
:1052F800C36A0BBFA260A160E160E2604BB12368A2
:1053080043F00E0323602B68002043F001032B6059
:10531800F0BD236823F004032360236843F00A03E5
:10532800F0E780F820600220F0BD000090F82130FE
:1053380010B5022B03D004238363012010BD03683A
:105348001A6822F00E021A601A6822F001021A6026
:10535800294A934224D902F56272934219D0143231
:10536800934218D01432934217D0143293420CBF90
:105378004FF480534FF48033204A536001230024B4
:1053880080F82130436B80F820409BB39847204633
:1053980010BD0123F0E71023EEE74FF48073EBE72D
:1053A80017498B4216D014318B4215D014318B42D9
:1053B80014D014318B4214D014318B4214D01431D0
:1053C8008B4214D0934214BF4FF480334FF0807354
:1053D8000C4AD2E70123FBE71023F9E74FF4807367
:1053E800F6E74FF48053F3E74FF48033F0E74FF4D8
:1053F8008013EDE7184610BD80000240000402400B
:10540800080002400000024070B40425C66B026C1C
:105418003468036895402542196855D04D0753D51F
:105428001A6896065EBF1A6822F004021A60604A7B
:1054380093421FD902F56272934214D014329342F8
:1054480013D01432934212D0143293420CBF4FF44B
:1054580080434FF48023574A5360C36A002B00F0FF
:10546800A58070BC18470423F5E74023F3E74FF401
:105478008063F0E750498B4216D014318B4215D027
:1054880014318B4214D014318B4214D014318B4216
:1054980014D014318B4214D0934214BF4FF480239C
:1054A8004FF08063454AD7E70423FBE74023F9E739
:1054B8004FF48063F6E74FF48043F3E74FF480231B
:1054C800F0E74FF48003EDE702259540254257D0D9
:1054D8008D0755D51A68940606D41A6822F00A0270
:1054E8001A60012280F82120314A93421ED902F520
:1054F8006272934213D01432934212D01432934200
:1055080011D0143293420CBF4FF400534FF40033C0
:10551800284A5360002380F82030836A9EE70223DC
:10552800F6E72023F4E74FF40073F1E722498B42B2
:1055380016D014318B4215D014318B4214D014314B
:105548008B4214D014318B4214D014318B4214D0B6
:10555800934214BF4FF400334FF00073174AD8E753
:105568000223FBE72023F9E74FF40073F6E74FF433
:105578000053F3E74FF40033F0E74FF40013EDE77F
:1055880008259540254211D009070FD5196821F043
:105598000E011960012303FA02F27260836380F836
:1055A8002130002380F82030036B57E770BC704728
:1055B800800002400004024008000240000002404F
:1055C8002DE9F74F002426466C4F6D4BDFF8B8E104
:1055D800DFF8B8C10A6832FA06F502D103B0BDE8AF
:1055E800F08F4FF0010808FA06F802EA0802904521
:1055F80040F084804D68122D00F0B18000F2878061
:10560800022D00F0A9807BD8002D00F08C80012DA0
:1056180000F0A0804FF00F09FF2A93BF824606F1E1
:105628008045083DD0F800B092BFB500D0F804B06E
:10563800AD0009FA05F82BEA080804FA05F588BF51
:1056480000F1040A48EA0505CAF80050D1F804A098
:105658001AF0805F52D0BD6926F0030845F00105B5
:10566800BD61BD6908F1804805F00105019508F59F
:10567800803806F0030B019D4FEA8B0BD8F80850D1
:1056880009FA0BF925EA09093E4DA8426CD005F53F
:105698008065A8426AD005F58065A84268D005F5FE
:1056A8008065A84266D005F58065A84264D070453B
:1056B8000CBF0525062505FA0BF545EA0905C8F8C6
:1056C80008501D681AF4803F14BF154395431D60A8
:1056D8005D681AF4003F14BF154395435D609D68EB
:1056E8001AF4801F14BF154395439D60DD681AF4B2
:1056F800001F14BF2A4325EA0202DA60013669E76F
:10570800032D25D0112D85D1CC68043482E7654559
:1057180009D012D8DFF878904D4504D009F58039C2
:105728004D457FF477AF8C68E4B1012C0CBFC0F80D
:105738001080C0F8148008246CE7DFF858904D45B5
:10574800F1D009F580394D45EDD0A9F58019E7E785
:1057580000245FE7CC685DE7CC6808345AE7CC687A
:105768000C3457E7042455E70025A4E70125A2E7F0
:105778000225A0E703259EE704259CE700100240C8
:105788000004014000080140001C014000002110F5
:1057980000001110000031100AB1016170470904BE
:1057A800FBE7C3680B4214BF416101617047000009
:1057B8002DE9F341054608B901203CE00368DB0701
:1057C80010D42B689F075DD42B68190700F19480CB
:1057D8002B685A0700F1BE80E869002840F02C8148
:1057E800002028E08F4C636803F00C03042B07D0DB
:1057F800636803F00C03082B09D16368DE0306D540
:1058080023689C03DDD56B68002BDAD1D4E76B687D
:10581800B3F5803F12D1236843F480332360FFF748
:10582800D9F9064623689803CBD4FFF7D3F9801B30
:105838006428F7D9032002B0BDE8F0819BB923683A
:1058480023F480332360236823F480232360FFF745
:10585800C1F9064623689903B3D5FFF7BBF9801B46
:105868006428F7D9E6E7B3F5A02F236803D143F4FA
:1058780080232360CFE723F480332360236823F455
:105888008023CBE7674C636813F00C0F07D063687D
:1058980003F00C03082B10D16368DA030DD42368D6
:1058A8009B0702D52B69012B86D123686A6923F0EF
:1058B800F80343EAC203236086E72A695A4B6AB1B0
:1058C80001221A60FFF786F9064623689F07ECD481
:1058D800FFF780F9801B0228F7D9ABE71A60FFF7BA
:1058E80079F90646236898077FF56EAFFFF772F9D6
:1058F800801B0228F6D99DE7AA694A4C4B4BDAB1BE
:1059080001221A60FFF766F90646636A9B070DD500
:105918004FF4FA52464B1B68B3FBF2F3019300BFF6
:10592800019B5A1E0192002BF9D151E7FFF752F95A
:10593800801B0228E9D97DE71A60FFF74BF9064674
:10594800636A9F077FF544AFFFF744F9801B02287D
:10595800F6D96FE7334CE369D80024D40127E3690B
:1059680043F08053E361E36903F080530093009BA5
:10597800304E3368D90518D5EB68012B26D1236A38
:1059880043F001032362FFF725F941F28836804688
:10599800236A9B073FD5002F3FF41EAFE36923F02E
:1059A8008053E36118E70027E2E7336843F4807324
:1059B8003360FFF70FF980463368DA05DCD4FFF768
:1059C80009F9A0EB08006428F6D933E7ABB9236AD4
:1059D80041F2883823F001032362236A23F0040389
:1059E8002362FFF7F7F80646236A9807D3D5FFF72F
:1059F800F1F8801B4045F7D91CE7052B236A03D132
:105A080043F004032362BAE723F001032362236A05
:105A180023F00403B6E7FFF7DDF8A0EB0800B04277
:105A2800B6D907E700100240000042428004424213
:105A380008020020007000402A4B5A681C4602F0F9
:105A48000C02082A3DD00023274E022833602BD1B0
:105A5800FFF7C0F80746236899011FD42B6AB3F5EE
:105A6800803F05D16268A96822F400320A43626067
:105A7800696A62680B4322F474121343636001235A
:105A88003360FFF7A7F8054623689A013FF5A8AEEB
:105A9800FFF7A0F8401B0228F6D9CBE6FFF79AF8E3
:105AA800C01B0228D7D9C5E6FFF794F80546236836
:105AB8009B017FF595AEFFF78DF8401B0228F6D9BC
:105AC800B8E601283FF4B7AE58682B6A00F4803274
:105AD8009A427FF471AE6B6A00F47010C01A18BF56
:105AE8000120A8E6001002406000424230B5194B80
:105AF80087B002AC03F110052246186859680833CC
:105B080003C2AB421446F7D101238DF804300223B7
:105B180011498DF805304B6803F00C02082A17D19B
:105B2800C3F3834206A80244DB0312F8102C0CD5F9
:105B38004B680A48C3F34043504306AA134413F87A
:105B4800143CB0FBF3F007B030BD05485043FAE70A
:105B58000248F8E7809F00080010024000127A000F
:105B680000093D002DE9F0410D46044610B9012019
:105B7800BDE8F081454A136803F007038B4229D337
:105B880021688E0731D4CA0744D4404A136803F009
:105B980007039D4267D322683D4D12F0040F6ED172
:105BA800130706D56B68226923F4605343EAC203DE
:105BB8006B60FFF79BFF6B68364AC3F30313D35C34
:105BC800D840354B1860354B1868FEF7C1FF0020E8
:105BD800BDE8F081136823F007030B4313601368D3
:105BE80003F007039942C2D1CAE7294B11F0040F09
:105BF8001EBF5A6842F4E0625A60080742BF5A68FA
:105C080042F460525A605A68A06822F0F0020243D7
:105C18005A60B8E762681E4E012A33681BD113F434
:105C2800003FA4D0736841F2883823F0030313437C
:105C38007360FEF7CFFF07467368626803F00C03D2
:105C4800B3EB820FA1D0FEF7C5FFC01B4045F3D9C7
:105C58000320BDE8F081022A02D113F0007FE0E7BB
:105C680013F0020FDDE7136823F007032B431360DB
:105C7800136803F007039D427FF479AF8BE76B68E5
:105C8800E16823F4E0630B436B6089E7002002407E
:105C98000010024082A00008080200200400002032
:105CA800044B054A5B68C3F30223D35C034A1068BC
:105CB800D84070470010024092A000080802002057
:105CC800044B054A5B68C3F3C223D35C034A1068DC
:105CD800D84070470010024092A000080802002037
:105CE80003682DE9F341D907054620D5354CE3690A
:105CF800DA0032D40127E36943F08053E361E369B2
:105D080003F080530193019B2F4E3368DB0526D5A2
:105D1800236A13F4407336D1236A6A6823F4407304
:105D2800134323621FB1E36923F08053E3612868BA
:105D3800830706D5234AA968536823F440430B43D5
:105D4800536010F010001BD01E4A69695368002088
:105D580023F480030B43536012E00027D4E7336831
:105D680043F480733360FEF735FF80463368D80507
:105D7800CED4FEF72FFFA0EB08006428F6D9032045
:105D880002B0BDE8F0816A6802F440729342C3D061
:105D980001200E4A236A1060002023F4407110602D
:105DA8002162D907B8D5FEF715FF41F288380646B3
:105DB800236A9A07B0D4FEF70DFF801B4045F7D938
:105DC800DDE700BF0010024000700040400442427E
:105DD80003680020DA6842F00102DA609A6802F08B
:105DE8000702062A1EBF1A6842F001021A607047AD
:105DF8007047704770477047036810B51A690446C2
:105E080091070ED5DA6892070BD56FF002021A6176
:105E180001229B6902779B0777D0FFF7EAFF0023EF
:105E2800237723681A69500710D5DA6851070DD50A
:105E38006FF004021A6102229B69227713F4407FF3
:105E4800204668D0FFF7D5FF0023237723681A6917
:105E580012070FD5DA6810070CD56FF008021A611F
:105E68000422DB692277990720465AD0FFF7C1FF41
:105E78000023237723681A69D20610D5DA68D0067A
:105E88000DD56FF010021A610822DB69227713F42E
:105E9800407F20464BD0FFF7ACFF002323772368D1
:105EA8001A69D10708D5DA68D20705D56FF001025B
:105EB80020461A6100F026FC23681A69100608D5E6
:105EC800DA68110605D56FF0800220461A6100F0E5
:105ED800BAF823681A69520608D5DA68500605D553
:105EE8006FF0400220461A61FFF785FF23681A69A0
:105EF800910622D5DA6892061FD56FF02002204657
:105F0800BDE810401A6100F09DB8FFF771FF204608
:105F1800FFF770FF83E7FFF76BFF2046FFF76AFF85
:105F280092E7FFF765FF2046FFF764FFA0E7FFF75A
:105F38005FFF2046FFF75EFFAFE710BD244A036806
:105F4800904212D002F5006290420ED0B0F1804F1C
:105F58000BD0A2F59832904207D002F580629042A9
:105F680003D002F5806290421DD14A6823F0700385
:105F78001343174A904212D002F5006290420ED0A5
:105F8800B0F1804F0BD0A2F59832904207D002F5BD
:105F98008062904203D002F58062904203D1CA68C1
:105FA80023F4407313434A6923F0800313430360C7
:105FB8008B68C3620B688362054B984203D003F574
:105FC8000063984201D10B69036301234361704761
:105FD800002C014010B50446A0B190F83D3003F004
:105FE800FF021BB980F83C2000F0D6FE022320688F
:105FF80084F83D30211DFFF7A1FF0123002084F81C
:106008003D3010BD012010BD90F83C3030B5012B5B
:106018004FF0020314D0046880F83D306268A3682A
:106028000D68496822F0700223F080030B432A436D
:106038006260A360012380F83D30002380F83C3083
:10604800184630BD704770470368DA6822F49072CA
:10605800DA605A6922F001025A61202380F83A3046
:106068007047000038B505460368C1681A691924E5
:1060780022F440520A431A6182680069D9680243CF
:10608800686921F4B05121F00C0102430A43DA6037
:106098005A69A96922F440720A435A610D4A934227
:1060A80014D1FFF70DFE60436C686422A400B0FBB6
:1060B800F4F0B0FBF2F402FB14031B013233B3FB20
:1060C800F2F3296803EB04138B6038BDFFF7E8FD92
:1060D800E9E700BF00380140F8B504460E46174608
:1060E8001D4621680B6836EA030301D10020F8BD7C
:1060F8006B1CF7D095B923680320DA6822F4D072B4
:10610800DA605A6922F001025A61202384F8393092
:1061180084F83A30002384F83830F8BDFEF75AFD89
:10612800C01B8542DDD2E6E710B5044640B390F8BF
:10613800393003F0FF021BB980F8382000F040FE28
:106148002423226884F83930D368204623F4005386
:10615800D360FFF787FF236800201A6922F4904272
:106168001A615A6922F02A025A61DA6842F4005226
:10617800DA602023E06384F8393084F83A3010BDBF
:10618800012010BD2DE9F0411F4690F83930044632
:10619800202B0D4690464ED1002949D0002A47D0E1
:1061A80090F83830012B46D0012380F8383000238E
:1061B800C363212380F83930FEF70CFD0646A4F8A6
:1061C8002480A4F82680E38C9BB26BB93B46324608
:1061D80040212046FFF780FFA8B9202384F8380023
:1061E80084F83930BDE8F081E38C3246013B9BB23C
:1061F800E384A3688021B3F5805F20463B460ED137
:10620800FFF76AFF10B10320BDE8F0812B882268F0
:10621800C3F308035360236943B90235D3E7FFF793
:106228005BFF0028EFD123682A785A600135CAE756
:106238000120BDE8F0810220BDE8F08138B50446B0
:10624800134694F83920202A2AD139B333B394F865
:106258003820012A24D00122002584F83820212260
:10626800E384206BE56384F839200E4AA384216215
:1062780082620D4A4563C2620C4A02632268043294
:10628800FFF716F86FF04002236828461A605A692B
:1062980084F8385042F080025A6138BD012038BD78
:1062A800022038BD4B630008796300084564000884
:1062B800134690F83A2073B5202A054638D10029AC
:1062C80034D0002B32D090F83820012A30D0012267
:1062D800002480F83820222281628385C46380F8F4
:1062E8003A20406B134A2E688262134A4463C262A2
:1062F800124A02630A46311DFEF7DAFF20462B6870
:1063080001941A6801925A6885F838400192019AF6
:10631800DA6842F48072DA605A6942F001025A611E
:106328005A6942F040025A6102B070BD0120FBE791
:106338000220F9E78363000839640008456400080F
:10634800704708B50368426A1B6813F020030AD136
:10635800D38413685A6922F080025A61DA6842F0DD
:106368004002DA6008BD1046FFF7EAFF08BD704733
:1063780008B5406AFFF7FBFF08BD08B50368426A25
:106388001B6813F0200310D1D3851368D96821F452
:106398008071D960596921F001015961596921F069
:1063A80040015961202382F83A30104600F0D6FEA9
:1063B80008BD90F83A3010B5222B36D183680169B0
:1063C800B3F5805F0268836A23D15268E9B9C2F3E2
:1063D800080223F8022B8362C48D013CA4B2C48551
:1063E8008CB90368DA6822F02002DA60DA6822F4ED
:1063F8008072DA605A6922F001025A61202380F81B
:106408003A3000F0ABFE002010BDD2B223F8012BC9
:10641800E1E721B9591C526881621A70DCE75268B9
:10642800591C816202F07F02F7E7022010BD704715
:1064380008B5406AFFF7FBFF08BD7047416A08B519
:106448000B685A6991F8390021280AD1120608D533
:106458000022CA84DA6822F0C002DA60202281F8B9
:1064680039205B6991F83A20222A06D15B0604D5C7
:1064780000230846CB85FFF7E7FDCB6B084643F0C2
:106488001003CB63FFF7D9FF08BD0000036870B5A0
:106498001A6804461607D9685D6907D196065AD561
:1064A8008D0658D5BDE87040FFF783BF15F001058C
:1064B80002D111F4907F4ED0D30705D5CE0542BF47
:1064C800E36B43F00103E363500704D51DB1E36BAD
:1064D80043F00203E363930704D51DB1E36B43F074
:1064E8000403E363160704D51DB1E36B43F0080307
:1064F800E363E36B002B66D0950604D5880602D5C6
:106508002046FFF756FF236820465D69E26B1107B6
:1065180002D415F040051AD0FFF796FD23685A6992
:10652800520610D55A69606B22F040025A6150B188
:10653800254B4363FEF7FAFE002844D0606BBDE8A4
:106548007040436B18472046FFF777FF70BDFFF791
:1065580074FFE56370BD160627D50D0625D594F89A
:106568003920212A2FD1A268B2F5805F226A17D17B
:106578001188C1F308015960216979B90232226290
:10658800E28C013A92B2E284EAB9DA6822F0800237
:10659800DA60DA6842F04002DA6070BD0132EEE794
:1065A800511C216212785A60EAE750060BD54A0658
:1065B80009D5DA68204622F04002DA60202384F800
:1065C8003930FFF7BDFE70BDD565000808B500235A
:1065D800406AC385C384FFF730FF08BD002310B5A8
:1065E8000F4CC90007290FDC61B141F2210213F4F5
:1065F800004F4FEA43039BB201F1FF3118BF5340EC
:106608000029F4D1184610BD10F8012B083982EA88
:10661800132234F8122082EA03239BB2E2E700BF78
:106628000800002010B59AB06422002101A800F0EB
:106638001DFE294B294C1A7812B12278032A08D852
:1066480001221A702378032B25D8DFE803F0262FC0
:1066580032351021224800F0B1FD4FF47A70FEF770
:10666800BFFA00F079F81F49024601A801F0AEFB15
:1066780001A8FDF7D5FDC1B201A800F09FFD01A852
:10668800FDF7CEFD01A9C2B2174801F059FA4FF43F
:10669800FA70FEF7A5FA1AB010BD0D21134800F0E4
:1066A8008DFD23780133DBB22370F4E70D21104808
:1066B800F5E71D210F48F2E715210F4800F07EFD90
:1066C8000520FEF78DFA0A210C4800F077FD0C48EA
:1066D80001F0BEFAE5E700BFF8030020F903002047
:1066E8009B9F0008B99F0008AC9F0008BC9F00084A
:1066F800CA9F0008D89F0008F69F00080CA0000851
:1067080017A0000802680A4B9A420FD1094A136879
:1067180001331360084A136801331360074A13688A
:1067280001331360064A136801331360704700BFD2
:106738000010004008040020040400200004002089
:10674800FC03002010B514460A230248FFF71AFD7F
:10675800204610BDF4050020014B1888704700BF83
:106768001C04002010B596B0282200210CA800F0C7
:106778007DFD1422002101A800F078FD18220021D7
:106788000DEB020000F072FD012310931023022488
:1067980011934FF460130CA815930C941394FFF7FE
:1067A80007F80F234FF4806201930023214601A8C4
:1067B8000393049205930294FFF7D4F94FF400432E
:1067C80006A806940893FFF78BFA16B010BD0000D0
:1067D8002DE9F04FBD4A8FB05168106807AB03C36D
:1067E8001189927ABA4D19809A70FEF7D5F9FFF798
:1067F800B9FF102200210AA800F038FDAB69002279
:1068080043F01003AB61AB6949F2400103F0100398
:106818000393039BAB69AF4843F00403AB61AB69D7
:10682800002403F004030493049BAB69012643F09E
:106838000803AB61AB69022703F008030593059BC6
:10684800AB694FF4602843F02003AB61AB694FF0AC
:10685800090B03F020030693069BFEF79DFF002219
:106868004EF2F2019C48FEF797FF002248F2D80149
:106878009A48FEF791FF002204219948FEF78CFF01
:1068880049F240030AA993480A930B960D970C9472
:10689800FEF796FE4EF2F2030AA98F480A930B966A
:1068A8000D970C94FEF78CFE48F2D8030AA98B4882
:1068B8000A930B960D970C94FEF782FE04230AA9FF
:1068C80087480A930B960D970C94FEF779FE6B692F
:1068D800844F33436B616B69834D33400293029B52
:1068E800824B28462B602E73C5F81C802E61AC6045
:1068F8002C756C600A940B940C94FEF7A3FB072389
:106908000AA92846CDF828B00B960C93FEF72EFA64
:10691800774B38463B60C7F81C803E61BC603C73CF
:106928003C757C600A940B940C94FEF78BFB0A234D
:106938004FF00B090AA938466E4F0A930B960C9430
:10694800FEF714FA6C4B38463B60C7F81C803E6172
:10695800BC603C733C757C600A940B940C94FEF705
:1069680071FB0AA93846CDF828900B960C94FEF7CF
:10697800FDF941F6FF03DFF89CA1604A50468AE81A
:106988000C00CAF80CB00A940B94CAF80840CAF86C
:106998001840FFF71FFB0AA95046DFF87C810A94CC
:1069A8000B94FFF731FB564B4FF00C0BC8F8003037
:1069B8004FF4E133534F4046C8F804300193C8F808
:1069C8000840C8F80C40C8F81040C8F814B0C8F817
:1069D8001840C8F81C40FFF7A7FB4B4A019B3846F4
:1069E8003A607B60BC60FC603C61C7F814B0BC6175
:1069F800FC61FFF799FB019B4448454A43600260EC
:106A08008460C4600461C0F814B08461C461FFF795
:106A18008BFB224621461020FEF7B2FB1020FEF722
:106A2800E3FB224621460F20FEF7AAFB0F20FEF7C4
:106A3800DBFB224621460E20FEF7A2FB0E20FEF7C6
:106A4800D3FB224621461120FEF79AFB1120FEF7C0
:106A5800CBFB224621462F20FEF792FB2F20FEF784
:106A6800C3FB224621463420FEF78AFB3420FEF77A
:106A7800BBFB224621463620FEF782FB3620FEF776
:106A8800B3FB224621461220FEF77AFB1220FEF7BE
:106A9800ABFB224621462520FEF772FB2520FEF798
:106AA800A3FB224621462620FEF76AFB2620FEF796
:106AB8009BFB224621464846FEF762FB4846FEF706
:106AC80093FB5046FFF784F928E000BF909F000829
:106AD800001002400010014000080140000C014075
:106AE80000140140980400200C05002000240140F7
:106AF800002801403C050020003C014000100040F7
:106B080000380140F806002000440040B806002084
:106B1800004C004078060020F4050020384B214640
:106B28001B68986801F09CF8364801F091F84946CE
:106B380007A8FFF753FD0146334801F001F8334930
:106B4800404600F0D1FA3846314900F0CDFA3246D5
:106B580029A7D7E9006728462E49FEF7C3F92E4D25
:106B6800DFF8C8902B68642B05D902214846FEF748
:106B780018FE00232B60294C2368B3F57A7F03D9CC
:106B8800FFF750FD0023236040F6B833DFF8A080FC
:106B9800D8F800209A4218D91E4B21481C6801F0E9
:106BA80057F8A4B221461F4800F0CAFF2046FDF757
:106BB80091FC32463B46FDF7F3FC02460B461A4869
:106BC80000F0BEFF0023C8F80030104CDFF86480E6
:106BD800A368002B09DC0E4CDFF85C80A368002B4F
:106BE800C0DD404600F098FAF8E7404600F094FA15
:106BF800EEE700BFAFF30080B4D934E70C684A3F32
:106C08000C0200202EA000083BA000083807002036
:106C1800440B00201C040020040400200004002071
:106C28004EA0000860A0000871A0000800080140FC
:106C3800FC030020F4050020F8060020704700003F
:106C48000E4B82B09A6942F001029A619A6902F089
:106C580001020092009ADA6942F08052DA61DB6937
:106C6800074A03F080530193019B536823F0E063C4
:106C780043F08063536002B0704700BF00100240C9
:106C88000000014030B505468BB01022002106A84F
:106C980000F0ECFA2B68384A934235D1374B384824
:106CA8009A6906A942F400729A619A69354C02F40D
:106CB80000720092009A9A6942F008029A619B69F0
:106CC80003F008030193019B022306930323079310
:106CD800FEF776FC8022E2604FF4007222614FF4E6
:106CE8000062294B626123602022002320466360F2
:106CF800A360A261E361FEF79BFA08B1FFF79EFF6C
:106D08002C6265620BB030BD204A93421BD11B4BED
:106D18009A6942F480629A619A6902F480620292E6
:106D2800029A9A6942F010029A619B6903F0100373
:106D38000393039B01230693032306A9144807938F
:106D4800FEF73EFCDEE7134A9342DBD10B4B9A6910
:106D580042F400429A619A6902F400420492049A49
:106D68009A6942F010029A619B6903F01003059337
:106D7800059B0223DFE700BF00240140001002400A
:106D8800000C0140340600200800024000280140A1
:106D980000100140003C01400268084B82B09A4252
:106DA8000AD103F50033DA6942F01002DA61DB69CF
:106DB80003F010030193019B02B0704700100040DC
:106DC80070B505468AB01022002106A800F04EFAD8
:106DD8002B68604A934229D15F4B06A9DA695F485C
:106DE80042F40022DA61DA6902F400220092009A81
:106DF8009A6942F010029A619B6903F010030193AB
:106E0800019B4FF48063069302230793032309939E
:106E1800FEF7D6FB4FF400630693002306A94F48FC
:106E280007930893FEF7CCFB0AB070BD4C4A934217
:106E380050D1494B06A99A694A4842F480429A615E
:106E48009A69002602F480420292029A9A69464C94
:106E580042F004029A619B6903F004030393039BC5
:106E68004FF4007306930223079303230993FEF755
:106E7800A7FB4FF480633B4806A90693079608963C
:106E8800FEF79EFB394B204684E848008023A66025
:106E9800E36026616661A661E661FEF7C9F908B19B
:106EA800FFF7CCFE6C636562314B324C23601023D4
:106EB800802263600023E260A36023616361A361B1
:106EC800E3612046FEF7B4F908B1FFF7B7FE2C637B
:106ED8006562A9E7284A9342A6D11F4B06A9DA6939
:106EE800204842F40032DA61DA69002602F40032FE
:106EF8000492049A9A69214C42F004029A619B69AF
:106F080003F004030593059B0423069302230793C8
:106F180003230993FEF754FB0823124806A9069396
:106F280007960896FEF74CFB154B204684E8480068
:106F38008023A660E36026616661A661E661FEF7CC
:106F480077F908B1FFF77AFE6C6365620D4B0E4C5A
:106F5800ACE700BF004C00400010024000100140A8
:106F680000380140000801406C050020580002402C
:106F780044000240C804002000440040540400209B
:106F88006C00024080000240B00500207047FEE718
:106F9800FEE7FEE7FEE7704770477047FDF70EBE55
:106FA8000148FEF731BA00BF340600200148FEF759
:106FB8002BBA00BFC80400200148FEF725BA00BF5D
:106FC8006C0500200148FEF71FBA00BF54040020DA
:106FD8000148FEF719BA00BFB005002008B50448FB
:106FE800FDF73FFEBDE808400248FDF73ABE00BF86
:106FF8000C050020980400200148FFF747BA00BF9D
:10700800F40500200148FFF741BA00BFF806002048
:107018000148FDF726BE00BF3C0500200148FFF7E8
:1070280035BA00BFB80600200148FEF7E5BE00BF2C
:107038007806002070B50E4615460C46A31B9D42E7
:1070480001DC284670BDAFF3008004F8010BF5E7BA
:1070580008B50A4B0246196809B909491960694611
:10706800186802448A4206D900F0D6F80C23036057
:107078004FF0FF3008BD1A6008BD00BF0C040020A7
:10708800540F00204FF0FF3070474FF4005300209A
:107098004B60704701207047002070470E4B1A68FC
:1070A80042F001021A6059680C4A0A405A601A688C
:1070B80022F0847222F480321A601A6822F4802244
:1070C8001A605A6822F4FE025A604FF41F029A604E
:1070D800034A044B9A607047001002400000FFF812
:1070E8000040000800ED00E0002330B40568074CBC
:1070F8004B600B608B600648064B012285420CBF33
:107108002046184630BC0C31FFF7D2B8F8060020EC
:1071180000440040F405002010B501680C4B0D4AEE
:107128000D4C914218BF1C4663682344187B00F03D
:107138001FFD636801200133B3F5806FA8BF0023EA
:107148006360A368013BA360BDE81040FDF748BD3C
:107158003807002000440040440B002038B502687E
:10716800114B124C9A42124B124D08BF1C46124B3F
:1071780008BF1D4623680133B3F5806FA8BF0023FD
:107188002360A3680133B3F5806FA36001DBFFF7C9
:10719800C3FF236804F10C0119442846BDE83840B0
:1071A8000122FFF785B800BF0044004038070020DF
:1071B800440B0020F4050020F80600200A4601468A
:1071C8000148FFF73BB800BFF8060020002103E0A4
:1071D8000B4B5B58435004310A480B4B42189A42F8
:1071E800F6D30A4A02E0002342F8043B084B9A42CD
:1071F800F9D3FFF753FF00F015F8FFF7E9FA7047E6
:1072080068A3000800000020DC030020DC03002045
:10721800540F0020FEE70000014B1868704700BFBC
:107228000C02002070B500250C4E0D4CA41BA410B8
:10723800A54209D102F092FE00250A4E0A4CA41B71
:10724800A410A54205D170BD56F8253098470135E0
:10725800EEE756F8253098470135F2E760A30008B5
:1072680060A3000860A3000864A300080346024462
:10727800934200D1704703F8011BF9E7002B2DE971
:10728800F0471E46BBBF03F100431E4600232D23D3
:1072980088B0149F129927F02007462F1446109D96
:1072A800DDF84CA00B7004D0452F00D10135022326
:1072B80000E0032307AA049206AA03928DE8280493
:1072C8002246334600F0F4FE472F804602D1119B38
:1072D800DB0726D5462F08EB050911D198F80030B1
:1072E800302B0AD10022002320463146FDF7C0FB8F
:1072F80018B9C5F10105CAF80050DAF80030994408
:107308000022002320463146FDF7B2FB38B930226F
:10731800079B994505D9591C07911A70F8E7CDF8CC
:107328001C904046079B159AA3EB0803136008B00E
:10733800BDE8F0870346F7B5002903F8022BB6BF6E
:107348002D222B2249420929427021DD0DF1070225
:1073580017460A2691FBF6F506FB1511092D01F1D2
:10736800300102F8011C02F1FF34294609DC3031F2
:10737800023A04F8011CBA421C4604D3201A03B08E
:10738800F0BD2246E6E712F8011B03F8011BF2E7FD
:1073980030221C46114404F8022B5970EEE7000015
:1073A8002DE9F04F91B00C461A9F93461E460546AC
:1073B80001F0CEFD036818460993FCF731FF00235E
:1073C8000E933B680A90073323F0070303F1080282
:1073D80094F81880D4F800A03A60D3E90023C4E9EF
:1073E8001223D4F84C90A76C29F000430B934FF06C
:1073F800FF32A64B38460B99FDF76CFB002840F08E
:10740800F7814FF0FF32A14B38460B99FDF744FB4B
:10741800002840F0ED810022002338464946FDF758
:1074280031FB10B12D2384F84330994B994FB8F1B3
:10743800470F98BF1F4603234FF0000923612AF026
:107448000403236000965B460FAA2146284600F0F5
:10745800DFF9013040F09A804FF0FF3011B0BDE8FD
:10746800F08F62680EA8531C0DF1340E4AF4806345
:1074780041D10622626000212360019363680DF107
:1074880033020590029200933A464B460691CDF896
:107498001080CDF80CE02846FFF7F0FE08F0DF0377
:1074A800472B074609D10D9BD81C02DB6268934223
:1074B80059DDA8F102085FFA88F8B8F1650F0D994F
:1074C80036D80139424604F150000D91FFF732FFDA
:1074D8000E9A81468318012A236102DC2268D107AB
:1074E80001D5013323619DF83330002BAAD02D2319
:1074F80084F84330A6E7B8F1670F02D0B8F1470F18
:10750800B9D19AB1002106910DF133018DE80C0033
:10751800236005903A46CDF81080CDF80CE0029132
:107528004B462846FFF7AAFE0746BCE70122A1E71B
:10753800B8F1660F19D1002963680CDD216113B910
:107548002268D20702D501330B4423610D9B4FF00B
:107558000009A365C7E713B92268D00701D502332C
:10756800F3E70123F1E74FF067080D9B0E9A93426A
:1075780005DB22682361D107E8D50133E5E7002B55
:10758800CCBF0123C3F102031344DEE723685A0585
:1075980007D423693A4659462846B04701302AD1CC
:1075A8005AE7B8F1650F40F2DC80D4E912010022F5
:1075B8000023FDF75DFA002839D00123364A5946E1
:1075C8002846B04701303FF447AF0E9B0D9A9A42C8
:1075D80002DB2368D8070ED50A9B099A5946284624
:1075E800B04701303FF438AF002704F11A080E9B6A
:1075F800013B9F4211DB23689F0708D5002704F150
:107608001908E3680F9A9B1A9F42C0F2E780E06866
:107618000F9B9842B8BF184620E7012342465946B7
:107628002846B04701303FF417AF0137DFE70D9B1D
:10763800002B33DC0123184A59462846B04701304D
:107648003FF40AAF0D9B23B90E9B13B92368D907E2
:10765800D1D50A9B099A59462846B04701303FF4CC
:10766800FBAE4FF0000804F11A090D9B5B429845E8
:1076780001DB0E9B8EE701234A4659462846B04750
:1076880001303FF4E9AE08F10108EEE7FFFFEF7FB4
:10769800A0A00008A4A00008B0A000080E9AA36D3E
:1076A8009A42A8BF1A46002A904636DC4FF0000AD4
:1076B80004F11A0328EAE8780B93D4F85890A9EB58
:1076C80008039A4531DB0E9B0D9A9A4238DB2368F2
:1076D800DA0735D40E9B0D99A3EB0902A3EB010839
:1076E8009045A8BF9046B8F1000F31DC002728EA82
:1076F800E87804F11A090D9A0E9B9B1AA3EB08036C
:107708009F42BFF678AF01234A4659462846B047FC
:1077180001303FF4A1AE0137EDE7134659463A462A
:107728002846B0470130C1D196E601230B9A594645
:107738002846B04701303FF48FAE0AF1010ABCE792
:107748000A9B099A59462846B0470130C2D183E6B8
:10775800434607EB090259462846B0470130C5D1D0
:107768007AE60E9A012A01DCDB0734D501233A4672
:1077780059462846B04701303FF46EAE0A9B099A35
:1077880059462846B04701303FF466AED4E91201A5
:1077980000220023FDF76CF950B1002704F11A0804
:1077A8000E9B013B9F420CDB4B4604F15002F2E674
:1077B8000E9B7A1C013B59462846B0470130F3D14D
:1077C8004AE60123424659462846B04701303FF46D
:1077D80043AE0137E4E701233A46ECE7012342468A
:1077E80059462846B04701303FF436AE013708E71E
:1077F8003A464B4638464946FDF76CF900283FF4AF
:1078080030AE014B014F12E6A8A00008ACA000085A
:107818002DE9F04791461F468A680B690646934250
:10782800B8BF1346C9F8003091F843200C46DDF87C
:10783800208012B10133C9F800302368990642BF8D
:10784800D9F800300233C9F80030256815F006056C
:1078580007D104F1190AE368D9F800209B1A9D4260
:107868002ADB94F843302268003318BF01239206BC
:107878002FD404F1430239463046C047013022D0A4
:107888002368E56803F00603042B18BF0025D9F820
:1078980000204FF0000908BFAD1AA368226908BF8D
:1078A80025EAE5759342C4BF9B1AED181A344D4575
:1078B8001BD10020BDE8F0870123524639463046E7
:1078C800C047013003D14FF0FF30BDE8F0870135E4
:1078D800C1E73020E11881F843005A1C94F845109C
:1078E8002244023382F84310C3E701232246394673
:1078F8003046C0470130E6D009F10109D7E700005A
:107908002DE9F04317460A7E85B06E2A984606464A
:107918000C460C9B01F1430E00F0BC801AD8632A78
:107928002ED00AD8002A00F0C880582A00F08A8091
:1079380004F1420584F842202AE0642A01D0692A29
:10794800F6D121681A6811F0800F23D0111D196033
:10795800136827E0732A00F0B48008D86F2A2AD069
:10796800702AE5D10A6842F020020A6003E0752A0D
:1079780021D0782ADCD178226F4984F8452064E048
:107988001A6801F14205111D1960136884F8423024
:107998000123A3E011F0400F02F104011960D7D0D0
:1079A800B2F90030002B03DA2D225B4284F8432021
:1079B80062490A2217E02068196810F0800F03D086
:1079C800081D18600B6806E010F0400F01F1040074
:1079D8001860F7D00B886F2A14BF0A22082257496B
:1079E800002084F843006568002DA560C0F29C80E3
:1079F800206820F004002060002B3FD1002D40F0CB
:107A080095807546082A0BD12368DA0708D52369BB
:107A180062689A42DEBF302305F8013C05F1FF3564
:107A2800AEEB05032361CDF800803B4603AA21464F
:107A38003046FFF7EDFE013055D14FF0FF3005B06D
:107A4800BDE8F08381F845203C492268186812F0A7
:107A5800800F00F104051D6001D0036802E055069F
:107A6800FBD50388D00744BF42F0200222601BB92F
:107A7800226822F0200222601022B1E77546B3FB8B
:107A8800F2F002FB1033CB5C05F8013D03460028F9
:107A9800F5D1B7E708681A6810F0800F496904D073
:107AA800101D18601368196007E010F0400F02F10C
:107AB800040018601368F6D0198000237546236106
:107AC800B1E71A68111D1960156800216268284617
:107AD80001F0B8FA08B1401B6060636823610023B5
:107AE80084F843309FE723692A4639463046C04721
:107AF8000130A2D023689B0707D5002504F1190996
:107B0800E368039A9B1A9D4205DBE068039B984251
:107B1800B8BF184693E701234A4639463046C0475E
:107B280001308AD00135EBE7002BA7D10B7804F19F
:107B3800420584F8423065E7C3A00008B2A00008F7
:107B48000FB40A4B13B51C6824B1A36913B92046B6
:107B580001F074F905AB049AA1682046019301F07D
:107B68008BFF02B0BDE8104004B070470C02002043
:107B780038B5084B05461C6824B1A36913B92046DB
:107B880001F05CF9A26829462046BDE8384002F0B9
:107B980089B800BF0C02002070B50E46054618B122
:107BA80083690BB901F04AF9AB69AC6813B9284687
:107BB80001F044F9234B9C4217D16C68A3891B0739
:107BC8001DD52369DBB1013EA36816F8011F013BEF
:107BD800A360E9B9002B2EDA22460A21284600F0D4
:107BE80019F9013011D00A2070BD174B9C4201D100
:107BF800AC68E3E7154B9C4208BFEC68DEE721461A
:107C0800284600F059F90028DDD04FF0FF3070BD4C
:107C1800002B04DAA269934206DB0A2904D0236800
:107C28005A1C22601970CFE72246284600F0F2F865
:107C38000130C9D1E9E70A2023685A1C226018706C
:107C480070BD00BF04A1000824A10008E4A000083A
:107C5800024B01461868FFF79FBF00BF0C020020C7
:107C680000294FF480630CBF0222002200F000B804
:107C78002DE9F7431D46514B04461E680F469046B2
:107C880026B1B36913B9304601F0D8F84C4B9C4281
:107C980052D17468B8F1020F06D0B8F1010F00F2A2
:107CA8008980002DC0F286802146304601F05CF8BC
:107CB800616B41B104F14403994202D0304601F0AE
:107CC800B9FC002363630023A3616360A3891B06D7
:107CD80003D52169304601F0ADFCA389B8F1020F44
:107CE80023F44A6323F00303A3815DD001AB6A4602
:107CF8002146304601F03AF9A3891843A0812DBBEB
:107D0800009D284601F096F9074600284ED1DDF877
:107D18000090A9453CD14FF0FF30A38943F00203FE
:107D2800A3810023A36004F1470323602361012397
:107D3800636103B0BDE8F083224B9C4201D1B46873
:107D4800A8E7214B9C4208BFF468A3E7002FD8D0CE
:107D5800B36913B9304601F071F8B8F1010F08BFE3
:107D6800A389276004BF43F00103A381A389276186
:107D780013F0080065611BD013F001004FF00003F9
:107D88001FBF6D42A360A561184608BFA560D0E774
:107D9800484601F04FF907460028BCD0A3894D4654
:107DA80043F08003A381D3E70020B6E7A946F5E7AF
:107DB800A060BEE74FF0FF30BBE700BF0C02002019
:107DC80004A1000824A10008E4A000080EB44FF4A0
:107DD800027100B59CB0ADF814106FF00041049129
:107DE80007914FF6FF711DAB02900690084853F8B3
:107DF800042BADF81610006802A9019301F020FDCC
:107E08000022029B1A701CB05DF804EB03B07047A7
:107E18000C020020F8B50E461446054618B18369D1
:107E28000BB901F00BF8214B9C422AD16C68A3696D
:107E3800A360A3891A072ED5236963B32369206831
:107E4800F6B2C01A63693746984204DB21462846D1
:107E580000F08AFF28BBA3680130013BA3602368B8
:107E68005A1C22601E706369984204D0A389DB07FC
:107E780019D50A2E17D12146284600F075FF90B172
:107E88000FE00B4B9C4201D1AC68D0E7094B9C42F8
:107E980008BFEC68CBE72146284600F00DF800281B
:107EA800CCD04FF0FF373846F8BD00BF04A100081A
:107EB80024A10008E4A00008324B70B51D680646EE
:107EC8000C4625B1AB6913B9284600F0B7FF2E4B15
:107ED8009C420FD16C68B4F90C309AB215072CD4B7
:107EE800D00611D40922326043F04003A3814FF039
:107EF800FF3070BD254B9C4201D1AC68EBE7244BA9
:107F08009C4208BFEC68E6E7510712D5616B41B1A6
:107F180004F14403994202D0304601F08BFB002360
:107F28006363A38923F02403A38100236360236987
:107F38002360A38943F00803A38123694BB9A3896C
:107F480003F42073B3F5007F03D02146304601F0D7
:107F580031F8A28912F001030CD00023A3606369F1
:107F68005B42A361236953B9B4F90C3013F0800064
:107F7800BAD170BD920758BF6369A360F2E70020C9
:107F8800F7E700BF0C02002004A1000824A10008A4
:107F9800E4A000082DE9F74F03690C6980469C426C
:107FA80000F38280013C01F1140700F1140657F830
:107FB800245056F824000135B0FBF5F54FEA840E3D
:107FC80006EB0E0307EB0E0901938DB34FF0000A81
:107FD8003846B446D34650F8042B93B205FB03A3A6
:107FE800120C4FEA134A05FB02A29BB2ABEB030348
:107FF800BCF800B04FEA124A5B441FFA82FBDCF877
:1080080000208145CBEB124202EB23429BB243EAAC
:1080180002434FEA224B4CF8043BDCD256F80E30B0
:1080280033B9019B043B9E421A4631D3C8F810402D
:10803800404601F028FA002826DB30464FF0000EB3
:10804800013557F8041BD0F800C08BB2AEEB030320
:108058001FFA8CF213440A0CC2EB1C4202EB2342B7
:108068009BB243EA0243B9454FEA224E40F8043B2B
:10807800E7D256F8242006EB84032AB9043B9E4233
:108088001A460BD3C8F81040284603B0BDE8F08F55
:108098001268043B002AC9D1013CC4E71268043BBA
:1080A800002AEFD1013CEAE70020EEE700000000DB
:1080B8002DE9F04F466A95B00446219DCDE902238B
:1080C8003EB9102000F0B6FF606246608660066028
:1080D800C660636A196851B15A68012393404A60BF
:1080E8008B60204600F0FBFF0022636A1A60039B46
:1080F800002BB7BF012300232B60039BAEBF2B606F
:1081080023F000430393DDF80C90AB4B33EA0903EB
:108118001BD142F20F73209A1360029B23B9C9F353
:108128001300002800F08385229B53B9A34B21E05C
:10813800A34B06930833229A1360069815B0BDE83E
:10814800F08F9E4B06930333F5E7DDE902670022C3
:10815800002330463946FCF78BFC804660B101238A
:10816800209A1360229B002B00F05E85954B229A83
:108178001360013B0693E0E712AB019313AB009346
:1081880032463B46204601F0F7F9C9F30A558246C4
:10819800002D7DD03046C7F3130343F07F5141F4DF
:1081A8004011A5F2FF35CDF840800022864BFCF740
:1081B80043F87BA3D3E90023FCF7F2F97AA3D3E9C8
:1081C8000023FCF73BF8064628460F46FCF782F9E1
:1081D80077A3D3E90023FCF7E3F902460B463046C0
:1081E8003946FCF72BF806460F46FCF789FC0022B7
:1081F8008346002330463946FCF744FC58B15846BC
:10820800FCF768F902460B4630463946FCF730FC65
:1082180008B90BF1FF3BBBF1160F58D8DDE9022373
:108228006A4901EBCB01D1E90001FCF749FC0028C0
:108238004FD000230BF1FF3B0D93129B5D1B6B1E70
:10824800079343BF0023C5F1010807934FF00008C7
:10825800BBF1000F3FDB079BCDF830B05B440793C1
:10826800002308931E9B092B00F2B480052BC4BF82
:10827800043B1E931E9BC8BF0026A3F10203D8BF70
:108288000126032B00F2B280DFE803F084862D7804
:10829800139B129D1D4405F23243202B11DD029AD7
:1082A80005F21240C3F1400322FA00F009FA03F381
:1082B8001843FCF7FFF80123A1F1F871013D109371
:1082C80073E7C3F12000029B03FA00F0F1E70123F2
:1082D800B2E70D90B1E7CBF1000308930023A8EBB8
:1082E8000B080C93BEE7012309931F9B002B40F357
:1082F80080809946049300220421656A6A6001F12E
:1083080014029A427AD96968204600F0B4FE636A7A
:1083180028601B68B9F10E0F069300F2F080002E5A
:1083280000F0ED80DDE90223BBF1000FCDE90E235B
:1083380079DD264A0BF00F034FEA2B1602EBC30335
:10834800F006D3E90023CDE90A235CD5DDE90E0167
:108358001F4B0325D3E90823FCF74CFACDE90201AA
:1083680006F00F061A4F002E4FD1DDE90A23DDE98A
:108378000201FCF73FFACDE902016EE001230993FF
:108388001F9B5B4403F1010904934B46012BB8BFC3
:108398000123B0E70023A7E70023F0E7AFF300804D
:1083A80061436F63A787D23FB3C8608B288AC63FF3
:1083B800FB799F501344D33F0000F07FDDA00008F5
:1083C800D4A00008B1A000080000F83F70A1000880
:1083D80048A100080126002309961E934FF0FF3399
:1083E80000220493994612231F9284E701230993DC
:1083F800F4E70123049399461A46F5E76A684900A9
:1084080001326A607BE70225ACE7F10708D5DDE9B0
:108418000A01D7E90023FCF7C3F8CDE90A010135C1
:10842800761008379FE700F0A580DDE90E01CBF153
:108438000006A24B06F00F0203EBC203D3E90023A8
:10844800FCF7AEF802250023CDE902019C4F361156
:10845800002E40F08480002B8DD10D9B002B00F066
:108468008B80DDE90223CDE90A23DDE90A01002238
:10847800944BFCF707FB00287ED0B9F1000F7BD0A6
:10848800049B002B37DDDDE90A0100228E4BFCF747
:1084980087F8CDE90201049E0BF1FF370135284624
:1084A800FCF718F8DDE90223FCF77AF8874B00227D
:1084B800FBF7C4FECDE90A010B9BA3F150750B95A0
:1084C800002E5CD1DDE902010022814BFBF7B4FEEE
:1084D8000A9A2B46CDE90201FCF7F2FA002840F08F
:1084E800F782DDE902010A9A05F10043FCF7CAFAAE
:1084F800002840F0EB82DDE90E23CDE90223139B2F
:10850800002BC0F25081BBF10E0F00F34C816B4B76
:1085180003EBCB03D3E90023CDE904231F9B002BF6
:1085280080F2DA80B9F1000F00F3D68040F0CD82F6
:10853800DDE904010022664BFCF732F8DDE902238D
:10854800FCF7B4FA4E464F46002840F0A482069B3A
:10855800069A5D1C31230BF1010B13709FE2F207A1
:1085680005D5D7E90023FCF71BF801230135761060
:1085780008376DE7022570E75F464E468FE7069A93
:108588004E4B32441192099A711E002A48D003EBCF
:10859800C103D3E9002300204E49FCF72BF9DDE99C
:1085A8000A23FBF749FECDE90A01069DDDE9020130
:1085B800FCF7A6FA0646FBF78DFF02460B46DDE9F7
:1085C8000201FBF739FEDDE90A23303605F8016BB5
:1085D800CDE90201FCF756FA002864D1DDE902234F
:1085E80000203849FBF728FEDDE90A23FCF74AFAA0
:1085F800002840F0B980119B9D423FF47CAFDDE933
:108608000A010022304BFBF7CBFF0022CDE90A011B
:10861800DDE902012C4BFBF7C3FFCDE90201C5E7F9
:1086280003EBC101D1E90001DDE90A23FBF7B8FF3B
:10863800CDE90A01069DDDE90201FCF761FA06466B
:10864800FBF748FF02460B46DDE90201FBF7F4FDA4
:108658003036119B05F8016BAB42CDE902014FF0B2
:10866800000224D11B4BDDE90A01FBF7E7FD0246B6
:108678000B46DDE90201FCF723FA002874D1DDE995
:108688000A2300201349FBF7D7FD02460B46DDE914
:108698000201FCF7F7F900283FF42DAF15F8013C6B
:1086A8006A1E302B01D0BB464DE01546F6E7064B57
:1086B800FBF776FFCDE90201BDE700BF70A1000816
:1086C80048A100080000F03F0000244000001C40C2
:1086D800000014400000E03F069DDDE90267DDE987
:1086E800042330463946FCF785F8FCF709FA80463A
:1086F800FBF7F0FEDDE90423FBF752FF02460B46C9
:1087080030463946FBF798FD08F1300605F8016B4D
:10871800069E0246AE1BB1450B4637D1FBF78EFDD0
:1087280006460F4602460B46DDE90401FCF7AAF9A6
:10873800C8B9DDE9040132463B46FCF799F910B1A6
:1087480018F0010F0FD15146204600F0C8FC002355
:10875800209A2B700BF101031360229B002B3FF42E
:10876800ECAC1D60E9E45F4615F8012C6B1E392A54
:1087780006D1069A9A4207D130231370134601375F
:108788001A7801321A708EE71D46EDE70022B54BC4
:10879800FBF706FF0022002306460F46FCF768F9A0
:1087A80000289CD0CFE7099A002A00F029811E9A58
:1087B800012A00F30E81109A002A00F0068103F2C4
:1087C80033434546089E079A01211A442046984497
:1087D800079200F024FD0746002D0BDD079B002BB8
:1087E80008DDAB42A8BF2B46079AA8EB0308ED1A91
:1087F800D31A0793089BFBB1099B002B00F0048157
:10880800002E11DD39463246204600F09DFD5246C5
:1088180001460746204600F00BFD51460A902046C7
:1088280000F05DFC0A9B9A46089B9A1B04D05146AF
:10883800204600F089FD82460121204600F0EFFC29
:108848000C9B0646002B40F3E1801A460146204661
:1088580000F07AFD1E9B0646012B40F3DA800023C8
:108868000893336906EB8303186900F08AFCC0F1AA
:108878002000079B184410F01F0000F0F080C0F1A2
:108888002003042B40F3E280079BC0F11C008044C6
:10889800054403440793B8F1000F05DD51464246ED
:1088A800204600F09FFD8246079B002B05DD3146E0
:1088B8001A46204600F096FD06460D9B002B00F058
:1088C800D3803146504600F0DEFD002880F2CC808F
:1088D800002351460A22204600F018FC099B0BF1A0
:1088E800FF3B8246002B00F0A981002339460A226B
:1088F800204600F00BFC049B0746002B03DC1E9B64
:10890800022B00F3B980002D05DD39462A462046A2
:1089180000F068FD0746089B002B00F0108179687D
:10892800204600F0A8FB05463A6907F10C0102321F
:1089380092000C3000F094FB01222946204600F0FA
:1089480051FD07970746029BDDF8188003F00103E5
:10895800089331465046FFF71DFB0799054600F17D
:108968003009504600F08FFD3A46029031462046C5
:1089780000F0A3FDC3680246002B40F0E2800146E8
:108988000990504600F07FFD0346099A114620469B
:10899800099300F0A4FB099B002B40F0D4801E9A99
:1089A800002A40F0D080089A002A40F0CC80B9F123
:1089B800390F00F0E880029B002B01DD05F1310939
:1089C80008F1010588F800906BE0129BC3F13603AB
:1089D800F7E6089B09F1FF36B342B7BF089B9E1B19
:1089E800F21A0C9BBFBF08969B180C930026B9F18E
:1089F800000FB9BFA8EB0905002345464B46E2E640
:108A0800089E4546099FE7E6089A10E71E9B012B3A
:108A180018DC029BB3B9039BC3F31303A3B9039BED
:108A280023F000431B0D1B052BB1079B08F1010820
:108A380001330793012308930C9B002B7FF411AF9C
:108A4800012016E70023F6E7029BF4E73FF423AF83
:108A5800079A1C331A4498441D4413461AE70346E0
:108A6800F6E700BF00002440B9F1000F33DC1E9B7D
:108A7800022B30DDCDF81090049B63B931460522F6
:108A8800204600F043FB01460646504600F0FBFC3A
:108A980000283FF75CAD1F9B069D6FEA030B002380
:108AA80007933146204600F01AFB002F3FF44BAEE7
:108AB800079B2BB1BB4203D01946204600F00FFBA1
:108AC8003946204600F00BFB3DE600263746E2E734
:108AD800BB4637463BE5099BCDF81090002B7FF449
:108AE80012AF069D31465046FFF754FA069B00F137
:108AF800300905F8019B049AEB1A9A4200F3818029
:108B0800069B012AACBF9B180133984600230793A4
:108B180051460122204600F065FC3146824600F0AD
:108B2800B2FC002834DC02D119F0010F30D14546DF
:108B380015F8013C6A1E302BB3D11546F8E73846C4
:108B4800FFE6012322E7029A002A04DB28D11E9AB5
:108B580032BB089A22BB002B7FF732AF5146012265
:108B6800204600F03FFC3146824600F08CFC00288D
:108B780005DC7FF425AF19F0010F3FF421AFB9F1FF
:108B8800390F7FF41BAF392308F1010808F8013CBD
:108B9800454615F8013C6A1E392B3AD001333FE0AF
:108BA800002B08F1010505DDB9F1390FEBD009F10A
:108BB800010907E7069B049AEB1A9342A84605F8B1
:108BC800019CA5D0514600230A22204600F09EFAB7
:108BD800079B8246BB424FF00A024FF000030799F9
:108BE800204604D100F092FA07900746B1E600F05B
:108BF8008DFA002307900A223946204600F086FAAB
:108C0800F3E7514600230A22204600F07FFA824605
:108C180068E7069B934205D13123069A0BF1010BB5
:108C280013703EE71546B4E7094BFFF7A3BA229B3A
:108C3800002B7FF47DAA074BFFF79CBA049B002BFF
:108C48003FF74FAF1E9B022B7FF74BAF14E700BFD8
:108C5800B0A00008D4A000088A892DE9F041054693
:108C680010070C465AD44B68002B05DC0B6C002B04
:108C780002DC0020BDE8F081E66A002EF9D000236E
:108C880012F480522F682B6033D0606DA3895A0785
:108C980005D56368C01A636B0BB1236CC01A002337
:108CA8000246E66A216A2846B047431CA38906D1D2
:108CB80029681D294BD82B4ACA40D60747D5002218
:108CC80062602269D904226004D5421C01D12B6854
:108CD80003B96065616B2F600029CAD004F14403B1
:108CE800994202D0284600F0A5FC00206063BDE848
:108CF800F081216A01232846B047411CC6D12B6860
:108D0800002BC3D01D2B01D0162B01D12F60B0E74B
:108D1800A38943F04003A381BDE8F0810F69002FC8
:108D2800A7D0930718BF00230E6808BF4B69A6EBAE
:108D380007080F608B60B8F1000F9ADD43463A468A
:108D4800216A2846A66AB047002807DCA38943F0B1
:108D58004003A3814FF0FF30BDE8F0810744A8EB42
:108D68000008E8E70100402038B50B6905460C46C5
:108D7800DBB118B183690BB900F060F80C4B9C4269
:108D880009D16C68B4F90C307BB121462846BDE89E
:108D98003840FFF761BF074B9C4201D1AC68F1E74F
:108DA800054B9C4208BFEC68ECE7002038BD00BFCB
:108DB80004A1000824A10008E4A00008014900F06B
:108DC800A9B800BF718D0008002310B504460360E0
:108DD8004360836081814366C2810361436183612B
:108DE800194608225C30FEF741FA054B246263629B
:108DF800044BA362044BE362044B236310BD00BF22
:108E0800399D00085B9D0008939D0008B79D0008E8
:108E180070B568254A1E55430E4605F1740100F0E9
:108E280055FC044640B1002180E842000C30A060A7
:108E380005F16802FEF71AFA204670BD836910B57D
:108E4800044633BB8364C3640365124B124A1B6830
:108E58008262984204BF0123836100F01FF86060BA
:108E6800204600F01BF8A060204600F017F800220A
:108E7800E06004216068FFF7A7FF01220921A068CC
:108E8800FFF7A2FF02221221E068FFF79DFF0123EE
:108E9800A36110BD9CA00008C58D0008F8B51C4B47
:108EA80007461E68B36913B93046FFF7C7FF48364F
:108EB800B4687368013B03D5336833B13668F7E7A4
:108EC800B4F90C506DB16834F4E704213846FFF763
:108ED8009FFF30600028F1D10C2304463B602046F8
:108EE800F8BD4FF6FF73E38101236566A381256012
:108EF800A560656025616561A5610822294604F1C0
:108F08005C00FEF7B3F96563A563A564E564E6E76D
:108F18009CA000082DE9F84380468946002600F108
:108F2800480414B93046BDE8F883A5686768013F6E
:108F380001D52468F5E7AB89012B07D9B5F90E30BF
:108F4800013303D029464046C84706436835EEE753
:108F5800044B1B68186A044B002808BF1846F030F9
:108F6800704700BF0C0200207002002070B50E464A
:108F7800B1F90E1090B0002914461D4607DA0023F7
:108F88002B60B3891A0610D44FF480630EE001AA4F
:108F980000F034FF0028F2DB029A02F47042A2F5D6
:108FA80000535A425A412A60EEE7402300202360CA
:108FB80010B070BD8B8973B59D0706460C4607D562
:108FC80004F14703236023610123636102B070BD8C
:108FD80001AB6A46FFF7CAFF00990546304600F024
:108FE80075FB48B9B4F90C309A05EFD423F00303A4
:108FF80043F00203A381E3E70D4BB362A38920602A
:1090080043F08003A381009B20616361019B5BB1F6
:10901800B4F90E10304600F003FF28B1A38923F0FD
:10902800030343F00103A381A3891D43A581CDE771
:10903800C58D0008024B0146186800F047BB00BF09
:109048000C02002010B5C9B202449042034601D177
:10905800002010BD1C7801308C42F6D1184610BD96
:1090680010B5431E0A44914200D110BD11F8014BBE
:1090780003F8014FF7E770B5456A04460E463DB957
:109088001020FFF7D7FF6062456085600560C56006
:10909800656AEB6883B1636ADB6853F82600B8B980
:1090A800012101FA06F56A1D9200204600F0B3FA84
:1090B80060B1466085600EE021220421204600F060
:1090C800AAFA636AE860DB68002BE4D1002070BD6F
:1090D800026843F8262000230361C36070BD70B5A1
:1090E800446A06460D463CB91020FFF7A3FF70629C
:1090F800446084600460C4603DB1736A6A68DB6878
:1091080053F82210296043F8225070BD2DE9F04130
:109118001F4606460C4600230D6901F1140EDEF8C1
:109128000000013381B202FB0171000C0F0C02FB3D
:10913800007089B201EB00419D424FEA10474EF89A
:10914800041BECDCD7B1A3689D4212DB6168304692
:109158000131FFF790FF8046226904F10C010232C9
:1091680092000C30FFF77CFF21463046FFF7B7FF2F
:10917800444604EB850301355F6125612046BDE85F
:10918800F081020C12040346B2B90304102013F054
:109198007F4F04BF1B02083013F0704F04BF1B0140
:1091A800043013F0404F04BF9B000230002B06DB55
:1091B8005B0003D5013070470020E8E720207047A6
:1091C8000368014613F007020BD0DA0723D4980787
:1091D80049BF5B089B0801200B605CBF0B60022045
:1091E800704798B2A8B910201B0C13F0FF0F04BFEA
:1091F8001B0A08301A0704BF1B0904309A0704BF6A
:109208009B080230DA0702D45B0806D001300B60F5
:1092180070471046E9E7002070472020704710B5D6
:109228000C460121FFF727FF01224461026110BDAE
:109238002DE9F74F14460A69236989469A42BEBF49
:109248000B46A1461C46D9F81070D4F810A0D9F8DE
:109258000830D9F8041007EB0A069E42C8BF01314E
:10926800FFF709FF00F114052B46002205EB8608DD
:10927800434516D304F1140209F1140102EB8A03E1
:1092880001EB87070193019C134694420CD8002EEA
:1092980003DD58F8043D002B54D0066103B0BDE847
:1092A800F08F43F8042BE3E7B3F800A00432BAF1D7
:1092B800000F20D0AE4689464FF0000C59F8044BF9
:1092C800BEF800B0A3B20AFB03B34FEA144BDEF8B2
:1092D800004063444FEA144C0AFB0BC404EB1344EC
:1092E8009BB243EA04434F454FEA144C4EF8043B03
:1092F800E4D8CEF800C032F8029CB9F1000F1FD0B4
:10930800AE468C464FF0000A2B68BCF80040BEF809
:1093180002B09BB209FB04B4A24443EA0A434EF8E4
:10932800043B5CF8043BBEF800401B0C09FB0343FC
:10933800674503EB1A434FEA134AE6D8CEF80030E4
:109348000435A0E7013EA2E72DE9F843154612F0DF
:10935800030206460F4607D0214C013A002354F871
:109368002220FFF7D3FE0746AD1035D0746A3CB90A
:109378001020FFF75FFE7062446084600460C46080
:10938800D6F82480D8F808404CB940F2712130460C
:10939800FFF745FF00230446C8F8080003604FF0B4
:1093A8000008EB070AD5394622463046FFF740FF4A
:1093B800814639463046FFF792FE4F466D100BD076
:1093C800206838B9224621463046FFF731FF206031
:1093D800C0F800800446E4E73846BDE8F88300BFDB
:1093E80038A200082DE9F0470C46074616462369BF
:1093F8004FEA621A0AEB03094968A36809F10105F3
:10940800AB4231DB3846FFF736FE00228046114674
:1094180000F1140352452ADB20692AEAEA7A04F1AA
:10942800140116F01F0203EB8A0301EB800E22D011
:109438000020C2F1200C0E689640304343F8040B1C
:1094480051F8040B8E4520FA0CF0F4D8186008B1D6
:1094580009F10205013D3846C8F810502146FFF7CA
:109468003EFE4046BDE8F08701315B00C8E743F89F
:1094780022100132CEE7043B51F8042B8E4543F805
:10948800042FF9D8E6E703690A6930B59B1A0CD1AD
:109498009200143014318418114454F8045D51F8C2
:1094A800042D954203D005D30123184630BDA042B0
:1094B800F3D3FAE74FF0FF33F7E72DE9F0470D460E
:1094C8000746114628461446FFF7DDFF061E08D159
:1094D80031463846FFF7CFFD012346610361BDE8F9
:1094E800F087A4BF23462C4638466168A6BF1D46B0
:1094F80000260126FFF7BFFD4FF0000CC6602B6960
:10950800266904F1140205F1140902EB860709EB38
:10951800830800F1140152F804AB59F8045B1FFAF0
:109528008AF36344ACB21B1B2C0CC4EB1A4404EB47
:1095380023449BB24FEA244CC84543EA0444964668
:1095480041F8044BE7D8BE4505D351F8043D8BB12B
:109558000661BDE8F0875EF8044BA2B262441314BA
:1095680003EB144392B242EA03424FEA234C41F818
:10957800042BE8E7013EE8E72DE9F3411C46012109
:109588009046089E099DFFF776FDC4F31302C4F3C5
:109598000A54074634BB0192B8F1000F27D002A83D
:1095A80040F8088DFFF70CFE0099F0B1019AC0F160
:1095B800200302FA03F30B43C2407B610192019B33
:1095C800002B14BF02210121BB613961C4B1A4F28F
:1095D800334404443460C0F135002860384602B092
:1095E800BDE8F08142F48012D5E77961E7E701A888
:1095F800FFF7E6FD0121019B39617B612030E5E73A
:10960800A0F2324007EB810330601869FFF7B9FD1B
:10961800C0EB4110E1E738B502FB01F4214600F048
:1096280055F8054618B122460021FDF71FFE2846C9
:1096380038BD000038B50546002943D051F8043C30
:109648000C1F002BB8BFE41800F038FC1E4A136842
:10965800104633B9636014602846BDE8384000F00E
:109668002EBCA3420BD921686218934201BF1A6825
:109678005B685218226063600460EDE713465A681D
:109688000AB1A242FAD919685818A0420BD1206829
:109698000144581882421960DED1106852680144AA
:1096A80019605A60D8E702D90C232B60D4E72068E8
:1096B80021188A4201BF1168526809182160626046
:1096C8005C60C9E738BD00BF1004002070B5CD1C30
:1096D80025F0030508350C2D38BF0C25002D06464E
:1096E80001DBA94203D90C233360002070BD00F0D0
:1096F800E5FB234A1468214691B9224C23681BB91B
:10970800304600F005FB20602946304600F000FB9B
:10971800431C26D10C233046336000F0D0FBE4E72D
:109728000B685B1B1AD40B2B0FD90B60CC18CD50D0
:10973800304600F0C4FB04F10B00231D20F00700A5
:10974800C31A1BD05A42E25070BD8C420BBF6368EB
:109758004B681360636018BF0C46E9E70C4649681C
:10976800CAE7C41C24F00304A04205D0211A3046DD
:1097780000F0CEFA0130CDD02560D9E770BD00BF2A
:1097880010040020140400202DE9F0478E6882465A
:109798009E420C469146984635D88A8912F4906FB5
:1097A80031D00223256809696F1A656905EB4505FB
:1097B80095FBF3F508F101033B449D4238BF1D4674
:1097C800530531D52946FFF781FF064650B90C23CA
:1097D800CAF80030A3894FF0FF3043F04003A3815B
:1097E800BDE8F0873A462169FFF73AFCA38923F4DC
:1097F800906343F08003A38126613E442660464679
:109808006561ED1BA560464528BF46464946324678
:10981800206800F039FBA36800209B1BA360236825
:109828001E442660BDE8F0872A4600F049FB06463C
:109838000028E1D121695046FFF7FCFEC7E7000088
:109848002DE9F04F9DB003938B8980461C060D4689
:1098580016460FD50B696BB94021FFF737FF286013
:10986800286128B90C23C8F800304FF0FF30C4E055
:1098780040236B610023099320238DF8293030237E
:109888004FF0010B8DF82A3037463C4614F8013B5F
:10989800002B3CD1B7EB060A0BD05346324629467B
:1098A8004046FFF771FF013000F0A280099B534446
:1098B80009933B78002B00F09B8000234FF0FF3288
:1098C80004930793059206938DF853301A93052253
:1098D80021785048FFF7B6FB671C049BD8B9D90616
:1098E80044BF20228DF853201A0744BF2B228DF83D
:1098F800532022782A2A16D000210A20079A2746C0
:109908003B780134303B092B50D9C9B111E0252BE4
:10991800C0D02746B9E73F4A3C46801A0BFA00F008
:1099280018430490D3E7039A111D12680391002A83
:1099380001DB079204E0524243F0020307920493CA
:109948003B782E2B0DD17B78791C2A2B32D1039BA7
:1099580002371A1D1B680392002BB8BF4FF0FF3364
:1099680005932D4C032239782046FFF76BFB38B15D
:109978004023001B03FA00F0049B013703430493C0
:109988003978062225487E1C8DF82810FFF75AFBE7
:10999800002835D0224BFBB9039B073323F007037C
:1099A80008330393099B4B4409936DE700FB02328C
:1099B8000121A4E700230A24184605930F463A78A4
:1099C8000131303A092A03D9002BCAD00590C8E7DB
:1099D80004FB00200123F1E703AB00932A46114B57
:1099E80004A94046FDF7DCFCB0F1FF3F8146D9D120
:1099F800AB895B063FF539AF09981DB0BDE8F08F1C
:109A080003AB00932A46074B04A94046FDF778FFAD
:109A1800EAE700BF44A200084AA200084EA20008D4
:109A2800A973000891970008936810B4013B002BB4
:109A3800936008DA9469A34202DBCBB20A2B02D105
:109A480010BCFEF7E7B91368581C10601970C8B24B
:109A580010BC7047F8B506460F461446D518AC42F8
:109A680001D1002007E03A4614F8011B3046FFF701
:109A7800DBFF431CF3D1F8BD2DE9F04F9DB00C4638
:109A880017460393064618B183690BB9FFF7D6F951
:109A98007C4B9C4257D17468A38918075DD523690C
:109AA800002B5AD00023099320238DF82930302326
:109AB8004FF0010B8DF82A30B846454615F8013BA2
:109AC800002B55D1B8EB070A0BD053463A4621462E
:109AD8003046FFF7BFFF013000F0C480099B5344B4
:109AE800099398F80030002B00F0BC8000234FF059
:109AF800FF3204930793059206938DF853301A9317
:109B0800052229786048FFF79DFA05F10108049BB2
:109B1800002831D1D90644BF20228DF853201A07D6
:109B280044BF2B228DF853202A782A2A2CD00021D2
:109B38000A20079AA84698F800300135303B092BCF
:109B48006DD971B326E0514B9C4201D1B468A3E7AB
:109B58004F4B9C4208BFF4689EE721463046FEF70B
:109B6800ABF900289ED04FF0FF301DB0BDE8F08F54
:109B7800252BA7D0A846A0E7434A4546801A0BFAEA
:109B880000F018430490BBE7039A111D1268039173
:109B9800002A01DB079204E0524243F002030792D5
:109BA800049398F800302E2B10D198F8013008F162
:109BB80001012A2B37D1039B08F102081A1D1B68E3
:109BC8000392002BB8BF4FF0FF330593314D0322AA
:109BD80098F800102846FFF735FA40B14023401B9B
:109BE80003FA00F0049B08F101080343049398F872
:109BF80000100622284808F101078DF82810FFF701
:109C080021FA002834D0254B03BB039B073323F0EC
:109C1800070308330393099B4B4409934CE700FB64
:109C28000232012186E700230A2518460593884653
:109C380098F800200131303A092A03D9002BC5D001
:109C48000590C3E705FB00200123F0E703AB009371
:109C58002246134B04A93046FDF7A2FBB0F1FF3FA3
:109C68008146D8D1A3895B063FF57DAF09987CE78B
:109C780003AB009322460A4B04A93046FDF740FE89
:109C8800ECE700BF04A1000844A2000824A10008D2
:109C9800E4A000084AA200084EA20008A973000820
:109CA8005D9A000870B50D461446064618B18369DA
:109CB8000BB9FFF7C3F8134B9C4212D17468A36821
:109CC800013B002BA36016DAA269934202DBEBB2D8
:109CD8000A2B10D1224629463046BDE87040FEF7CF
:109CE80099B8094B9C4201D1B468E8E7074B9C42FC
:109CF80008BFF468E3E72368E8B25A1C22601D70C5
:109D080070BD00BF04A1000824A10008E4A0000859
:109D180038B50023054C054608462360FDF798F939
:109D2800431C02D1236803B12B6038BD500F0020BB
:109D380010B50C46B1F90E1000F0E8F80028ABBFDA
:109D4800636DA3891B1823F48053ACBF6365A3819B
:109D580010BD2DE9F0411F468B890546DB050C46F1
:109D6800164605D502230022B1F90E1000F068F856
:109D7800A389324623F48053A381B4F90E103B46DD
:109D88002846BDE8F04100F017B810B50C46B1F907
:109D98000E1000F055F8431CA38915BF606523F425
:109DA800805343F48053A38118BFA38110BDB1F938
:109DB8000E1000F013B8000038B5054608461146E5
:109DC8000022054C22601A46FCF7BCFC431C02D159
:109DD800236803B12B6038BD500F002038B500232D
:109DE800054C054608462360FDF74CF9431C02D193
:109DF800236803B12B6038BD500F002038B500230D
:109E0800064C0546084611462360FDF73EF9431CFB
:109E180002D1236803B12B6038BD00BF500F00206A
:109E280038B50023054C054608462360FDF732F98E
:109E3800431C02D1236803B12B6038BD500F0020AA
:109E480038B50546084611460022054C22601A46D8
:109E5800FDF722F9431C02D1236803B12B6038BDFA
:109E6800500F002082B001B901A942B14BB113785B
:109E78000B601278101C18BF012002B07047104602
:109E8800FBE76FF00100F8E7884210B501EB020329
:109E980003D8421E99420CD110BD9842F9D28118BC
:109EA800D21AD34200D110BD13F8014D01F8014D6B
:109EB800F7E711F8014B02F8014FEBE770477047DD
:109EC800F8B5074614460E4621B91146BDE8F840D4
:109ED800FFF7FCBB22B9FFF7ADFB25462846F8BDC6
:109EE80000F033F884420FD921463846FFF7EEFBDD
:109EF80005460028F2D031462246FFF7B1F8314630
:109F08003846FFF797FBE9E73546E7E738B50546F2
:109F1800084611460022054C22601A46FDF78AF8C9
:109F2800431C02D1236803B12B6038BD500F0020B9
:109F380049B1FF2A8BBF8A230A700360012088BFBA
:109F48004FF0FF3070470846704751F8040C00285E
:109F5800A0F10400BCBF0B58C0187047F8B500BF8B
:109F6800F8BC08BC9E467047F8B500BFF8BC08BCF2
:049F78009E4670474A
:109F800002030405060708090A0B0C0D0E0F10103A
:109F9000000102030405060708090A41542B43493E
:109FA0005053454E443D302C340D0A0025730D0AA4
:109FB00020494E444558203A2025640041542B4303
:109FC000574D4F44453D330D0A0041542B434950F2
:109FD0004D55583D310D0A0041542B4357534150C4
:109FE0003D22424C55455F54455354222C22222C8D
:109FF000352C300D0A0041542B43495053455256DD
:10A0000045523D312C343030300D0A0041542B4341
:10A01000494653520D0A00455350205365747469E4
:10A020006E6720436F6D706C657465200D0055611F
:10A030007274205374617274200D00437263206740
:10A04000656E6572617465202578200D0A003D3DBE
:10A050003D3D3D3D3D3D3D3D3D3D3D3D3D3D3D006D
:10A060004144432056616C65203A202564200D0A46
:10A07000004144432056616C65203A202566200D3E
:10A080000A000000000000000000010203040607AF
:10A090000809000000000102030400001002002073
:10A0A000494E4600696E66004E414E006E616E007C
:10A0B0003000303132333435363738394142434459
:10A0C00045460030313233343536373839616263D2
:10A0D00064656600496E66696E697479004E614E0A
:10A0E0000000000000000000000000000000000070
:10A0F0000000000000000000000000000000000060
:10A10000000000000000000000000000000000004F
:10A11000000000000000000000000000000000003F
:10A12000000000000000000000000000000000002F
:10A13000000000000000000000000000000000001F
:10A1400000000000000000000080E03779C34143B8
:10A15000176E05B5B5B89346F5F93FE9034F384D8D
:10A16000321D30F94877825A3CBF737FDD4F157539
:10A17000000000000000F03F00000000000024404C
:10A1800000000000000059400000000000408F4027
:10A19000000000000088C34000000000006AF84092
:10A1A0000000000080842E4100000000D0126341B6
:10A1B0000000000084D797410000000065CDCD412C
:10A1C000000000205FA00242000000E8764837420D
:10A1D000000000A2941A6D42000040E59C30A242AB
:10A1E0000000901EC4BCD64200003426F56B0C4320
:10A1F0000080E03779C3414300A0D88557347643C7
:10A2000000C84E676DC1AB43003D9160E458E14327
:10A21000408CB5781DAF154450EFE2D6E41A4B449C
:10A2200092D54D06CFF08044F64AE1C7022DB544E1
:10A23000B49DD9794378EA44050000001900000074
:10A240007D000000232D302B2000686C4C006566DB
:10A2500067454647004300504F534958002E0000C1
:10A2600020202020202020202028282828282020C6
:10A2700020202020202020202020202020202020DE
:10A280008810101010101010101010101010101056
:10A290000404040404040404040410101010101036
:10A2A000104141414141410101010101010101010F
:10A2B0000101010101010101010101101010101043
:10A2C00010424242424242020202020202020202E0
:10A2D0000202020202020202020202101010102008
:10A2E000000000000000000000000000000000006E
:10A2F000000000000000000000000000000000005E
:10A30000000000000000000000000000000000004D
:10A31000000000000000000000000000000000003D
:10A32000000000000000000000000000000000002D
:10A33000000000000000000000000000000000001D
:10A34000000000000000000000000000000000000D
:10A3500000000000000000000000000000000000FD
:04A360000D420008A2
:04A36400E9410008C3
:10A3680001000000100000000000211042206330AE
:10A378008440A550C660E770088129914AA16BB155
:10A388008CC1ADD1CEE1EFF13112100273325222FD
:10A39800B5529442F772D662399318837BB35AA3A5
:10A3A800BDD39CC3FFF3DEE36224433420040114CD
:10A3B800E664C774A44485546AA54BB528850995F5
:10A3C800EEE5CFF5ACC58DD553367226111630069D
:10A3D800D776F6669556B4465BB77AA71997388745
:10A3E800DFF7FEE79DD7BCC7C448E5588668A7785D
:10A3F8004008611802282338CCC9EDD98EE9AFF995
:10A40800488969990AA92BB9F55AD44AB77A966A3C
:10A41800711A500A333A122AFDDBDCCBBFFB9EEBE4
:10A42800799B588B3BBB1AABA66C877CE44CC55C0C
:10A43800222C033C600C411CAEED8FFDECCDCDDD34
:10A448002AAD0BBD688D499D977EB66ED55EF44EDC
:10A45800133E322E511E700E9FFFBEEFDDDFFCCF84
:10A468001BBF3AAF599F788F8891A981CAB1EBA1D8
:10A478000CD12DC14EF16FE18010A100C230E32054
:10A488000450254046706760B9839893FBA3DAB3FC
:10A498003DC31CD37FE35EF3B1029012F322D232A4
:10A4A8003542145277625672EAB5CBA5A8958985CC
:10A4B8006EF54FE52CD50DC5E234C324A0148104F4
:10A4C8006674476424540544DBA7FAB79987B8979C
:10A4D8005FE77EF71DC73CD7D326F2369106B01644
:10A4E80057667676154634564CD96DC90EF92FE95C
:10A4F800C899E9898AB9ABA9445865480678276894
:10A50800C018E1088238A3287DCB5CDB3FEB1EFB3B
:10A51800F98BD89BBBAB9ABB754A545A376A167AE3
:10A52800F10AD01AB32A923A2EFD0FED6CDD4DCD0B
:10A53800AABD8BADE89DC98D267C076C645C454C33
:10A54800A23C832CE01CC10C1FEF3EFF5DCF7CDFDB
:10A558009BAFBABFD98FF89F176E367E554E745E83
:10A56800932EB23ED10EF01E0024F40010020020FB
:10A578000000000004A1000824A10008E4A00008CD
:10A5880000000000000000000000000000000000C3
:10A5980000000000000000000000000000000000B3
:10A5A80000000000000000000000000000000000A3
:10A5B8000000000000000000000000000000000093
:10A5C8000000000000000000000000000000000083
:10A5D8004300000000000000000000000000000030
:10A5E8000000000000000000000000000000000063
:10A5F8004300000000000000000000000000000010
:10A608000000000000000000000000000000000042
:10A6180043000000000000000000000000000000EF
:10A628000000000000000000000000000000000022
:10A6380043000000000000000000000000000000CF
:10A648000000000000000000000000000000000002
:10A6580043000000000000000000000000000000AF
:10A6680000000000000000000000000000000000E2
:10A67800430000000000000000000000000000008F
:10A6880000000000000000000000000000000000C2
:10A69800430000000000000000000000000000006F
:10A6A80000000000000000000000000000000000A2
:10A6B800399F00086D9E0008000000005FA2000896
:10A6C8005DA2000870A0000870A0000870A0000833
:10A6D80070A0000870A0000870A0000870A0000812
:10A6E80070A0000870A00008FFFFFFFFFFFFFFFF3A
:10A6F800FFFFFFFFFFFF00000100415343494900EE
:10A708000000000000000000000000000000000041
:10A7180000000000000000000000415343494900C8
:10A728000000000000000000000000000000000021
:0CA7380000000000000000000000000015
:04000005080071D5A9
:00000001FF
